:020000040000FA
:0400000069303A2801
:040004000034003490
:08000800A000030EA100831209
:1000100005191128831601178312B2308100B1012E
:100020002C2883160113831203140B190310A80D37
:10003000A90DAA0DAB0DAC0DAC16FF302C02031DA3
:100040002C28FA302B02031D2C2832152A08AF0069
:100050002908AE002808AD008B100B11210E83007B
:06006000A00E200E0900B5
:0C007400203084008001840A80300402E7
:10008000031C3C283F2283160C3085058701831210
:10009000850187010730990000309A0010308316DF
:1000A0008E008312603083168F0083120030831617
:1000B00091009F008312C830831681008312313073
:1000C0009000003083168C00831210308B00BD1B13
:1000D0006F2885196F286400851D6B28DB233D1C64
:1000E00072283C2381018E018F010B118B100B10A4
:1000F0008C018B178A20321996202122B40B882874
:10010000031085190314BA0DF0303A0203199E2129
:100110004D237A2864003310B10A311F9528AC01B1
:10012000AB01AA01A901A801B101080032110130F7
:10013000B70085144008013ECE000F08CF008B1396
:100140002030370783169B001C141A088312A40062
:100150001030370783169B001C141A088312A30063
:10016000A6000230A6060030370783169B001C1439
:100170001A088312A200A7000130A7068B17331CB0
:10018000C72822090339A200A309A409A509240844
:100190002F02031D982923082E02031D312922084E
:1001A0002D02031D982901303702031DDE283D1959
:1001B000DD283E18DE283E143F145C220230370250
:1001C000031DE9283D19E828BE18E928BE143F148C
:1001D000692203303702031DF4283D19F3283E1924
:1001E000F4283E153F14762204303702031DFF2801
:1001F0003D19FE28BE19FF28BE153F148322053085
:100200003702031D0A293D1909293E1A0A293E16FB
:100210003F14902206303702031D15293D19142979
:10022000BE1A1529BE163F149D2207303702031D42
:1002300020293D191F293E1B20293E173F14AA22C1
:1002400008303702031D2B293D192A29BE1B2B29F3
:10025000BE173F14B72209303702031D31293F145E
:10026000C42226082E02031D982927082D02031DEB
:10027000982901303702031D44293D1943293E1CAA
:1002800044293E103F14EB2202303702031D4F2950
:100290003D194E29BE1C4F29BE103F14EF220330DA
:1002A0003702031D5A293D1959293E1D5A293E116D
:1002B0003F14F32204303702031D65293D196429D8
:1002C000BE1D6529BE113F14F72205303702031DFC
:1002D00070293D196F293E1E70293E123F14FB22E2
:1002E00006303702031D7B293D197A29BE1E7B2962
:1002F000BE123F14FF2207303702031D86293D1925
:1003000085293E1F86293E133F14032308303702F8
:10031000031D91293D199029BE1F9129BE133F1439
:10032000072309303702031D97293F140B2398290F
:10033000B70A0A303702031808009F280130B600B8
:10034000B400B500B70085018701B2138A20B40B51
:10035000B929031085190314BA0DF0303A020319B4
:10036000E129B51F8510B50BB9299630B500FC21E0
:10037000F321321DA6293211331CC3292D0903395B
:10038000AD00AE09AF092F1CA6292D0830020319B4
:10039000A6292D08B0002E1EA6298B132030370762
:1003A000BC002F08BB002A2210303707BC002E08E3
:1003B000BB002A2200303707BC002D08BB002A22D0
:1003C0008B1785018701083037022030031985001B
:1003D0002A3003198700B70AB6010A303702031C16
:1003E000A6293C2308003708B6080319B6000319EC
:1003F00008008514B60308000130370203190F23E3
:10040000023037020319132303303702031917236D
:100410000430370203191B230530370203191F2349
:100420000630370203192323073037020319272325
:100430000830370203192B230930370203192F2301
:1004400008003F1C08003F101030BC003E08BB00F5
:100450002A2208008B133B0883161C159A0083126E
:100460003C0883169B0055309D00AA309D009C14CB
:1004700064009C18382A1C1183128B1708008316FD
:1004800000309B001C141A088312BD008316103024
:100490009B001C141A0883123D18BE0083162030DE
:1004A0009B001C141A088312C1000130C11BC1003B
:1004B000C1080319C10008003D19871640083D1DF9
:1004C00040034107D0000F08D100BD1936233E1468
:1004D00008003D19071640083D1D40034107D200A2
:1004E0000F08D300BD193623BE1408003D19871527
:1004F00040083D1D40034107D4000F08D500BD1939
:1005000036233E1508003D19051640083D1D4003E1
:100510004107D6000F08D700BD193623BE150800C5
:100520003D19851640083D1D40034107D8000F08BE
:10053000D900BD1936233E1608003D19071540089D
:100540003D1D40034107DA000F08DB00BD193623CB
:10055000BE1608003D19871440083D1D40034107A1
:10056000DC000F08DD00BD1936233E1708003D19D9
:10057000071440083D1D40034107DE000F08DF005F
:10058000BD193623BE170800BD1908003D1DCC2A31
:10059000303085043F3087048E018F01C001D001C7
:1005A000D201D401D6010130D800DA00DC00DE002F
:1005B0004030D1008030D300C030D500FF30D700AC
:1005C0004030D9008030DB00C030DD00FF30DF007C
:1005D000FF30BE00080087128E018F01080007124D
:1005E0008E018F01080087118E018F01080005120E
:1005F0008E018F01080085128E018F0108000711FE
:100600008E018F01080087108E018F0108000710EE
:100610008E018F01080036238E018F010800070824
:10062000203A870008000708103A870008000708EA
:10063000083A870008000508103A850008000508F8
:10064000203A850008000708043A870008000708D8
:10065000023A870008000708013A870008000508E9
:10066000303A850007083F3A87000800CF308505FB
:10067000C0308705BE0108003E188716BE18071651
:100680003E198715BE1905163E1A8516BE1A07159E
:100690003E1B8714BE1B071408003D19512B3E1C3E
:1006A0005D2B50084002031D5D2B51080F02031CF7
:1006B0005D2B3D1987123D1D87163D19612BBE1C10
:1006C0006D2B52084002031D6D2B53080F02031CB3
:1006D0006D2B3D1907123D1D07163D19712B3E1D4F
:1006E0007D2B54084002031D7D2B55080F02031C6F
:1006F0007D2B3D1987113D1D87153D19812BBE1D91
:100700008D2B56084002031D8D2B57080F02031C2A
:100710008D2B3D1905123D1D05163D19912B3E1ED1
:100720009D2B58084002031D9D2B59080F02031CE6
:100730009D2B3D1985123D1D85163D19A12BBE1E11
:10074000AD2B5A084002031DAD2B5B080F02031CA2
:10075000AD2B3D1907113D1D07153D19B12B3E1F4E
:10076000BD2B5C084002031DBD2B5D080F02031C5E
:10077000BD2B3D1987103D1D87143D19C12BBE1F90
:10078000CD2B5E084002031DCD2B5F080F02031C1A
:10079000CD2B3D1907103D1D07144E084002031DC7
:1007A000D62B4F080F02031CD62B85100C1C0800FB
:1007B0000C10C00A0800B601B401B5013D1CE32BC2
:1007C000BD01BD14EF2BBD1CE82BBD013D15EF2B6A
:1007D0003D1DED2BBD01BD15EF2BBD013D143D08A9
:1007E000B6006400F32BF42BF52BF62BF72BB51B7F
:1007F0008716B51F8712B40BF12BB50BF12B031025
:10080000B60CB608031DF12B0030BC003D08BB0040
:040810002A22080090
:0840000008000300060009009E
:02400E00CC33B1
:10420000010078007A007C007E007B0079007F004E
:104210007D007A0078007E007C00FF00FF00FF0038
:104220000000F200F600FA00FE00F200F600FA00CC
:10423000FE00F200F600FA00FE00FF00FF00FF00A3
:10424000010005000500050005000900090009003E
:1042500009000D000D000D000D00FF00FF00FF0024
:10426000FF00FF00FF00FF00FF00FF00FF00FF0056
:10427000FF00FF00FF00FF00FF00FF00FF00FF0046
:10428000FF00FF00FF00FF00FF00FF00FF00FF0036
:10429000FF00FF00FF00FF00FF00FF00FF00FF0026
:1042A000FF00FF00FF00FF00FF00FF00FF00FF0016
:1042B000FF00FF00FF00FF00FF00FF00FF00FF0006
:1042C000FF00FF00FF00FF00FF00FF00FF00FF00F6
:1042D000FF00FF00FF00FF00FF00FF00FF00FF00E6
:1042E000FF00FF00FF00FF00FF00FF00FF00FF00D6
:1042F000FF00FF00FF00FF00FF00FF00FF00DD00E8
:00000001FF
